:100000000C9458060C9475060C9475060C947506A1
:100010000C9475060C9475060C9475060C94750674
:100020000C9475060C9475060C9475060C94750664
:100030000C9475060C9475060C9475060C946F0E52
:100040000C9475060C9475060C9475060C945E0D54
:100050000C94C00D0C9475060C94EA0D0C94750666
:100060000C9475060C9475060C9475060C94750624
:10007000000000000000000000000000007EC381BE
:10008000A581BD99C37E0000007EFFFFDBFFC3E7B3
:10009000FF7E0000000044EEFEFEFE7C38100000F3
:1000A0000010387CFEFE7C381000000000183C3C3C
:1000B000FFE7E718187E000000183C7EFFFF7E185F
:1000C000187E00000000000000000000000000009A
:1000D0000000000000000000000000000000000020
:1000E0000000000000000000000000000000000010
:1000F00000000000003E0E3A72F8CCCCCC78000034
:10010000003C6666663C187E18180000000000007F
:100110000000000000000000007F637F63636367EE
:10012000E7E6C000000018DB7EE7E77EDB18000092
:100130000080C0E0F8FEF8E0C08000000002060E7B
:100140003EFE3E0E0602000000183C7E1818187E87
:100150003C18000000666666666600006666000081
:10016000007FDBDBDB7B1B1B1B1B0000007E633087
:100170003C66663C0CC67E0000000000000000FEED
:10018000FEFE000000183C7E1818187E3C187E0009
:1001900000183C7E181818181818000000181818B5
:1001A0001818187E3C180000000000180CFE0C18EF
:1001B000000000000000003060FE60300000000021
:1001C00000000000C0C0C0FE0000000000000024CD
:1001D00066FF6624000000000000101038387C7CA8
:1001E000FEFE00000000FEFE7C7C3838101000008F
:1001F00000000000000000000000000000307878DF
:100200007830300030300000006666662400000060
:1002100000000000006C6CFE6C6C6CFE6C6C0000EE
:1002200030307CC0C0780C0CF8303000000000C4C6
:10023000CC183060CC8C00000070D8D870FADECCBE
:10024000DC7600000030303060000000000000006C
:10025000000C183060606030180C0000006030182E
:100260000C0C0C1830600000000000663CFF3C667F
:100270000000000000000018187E181800000000A0
:10028000000000000000000038386000000000009E
:1002900000FE000000000000000000000000000060
:1002A00038380000000002060C183060C0800000E2
:1002B000007CC6CEDED6F6E6C67C0000001030F02C
:1002C0003030303030FC00000078CCCC0C1830607E
:1002D000CCFC00000078CC0C0C380C0CCC78000066
:1002E000000C1C3C6CCCFE0C0C1E000000FCC0C0C2
:1002F000C0F80C0CCC780000003860C0C0F8CCCC42
:10030000CC78000000FEC6C6060C18303030000065
:100310000078CCCCCC78CCCCCC7800000078CCCC9D
:10032000CC7C18183070000000000038380000380D
:10033000380000000000003838000038381830005D
:10034000000C183060C06030180C00000000000085
:100350007E007E0000000000006030180C060C18C3
:10036000306000000078CC0C1830300030300000D5
:10037000007CC6C6DEDEDEC0C07C0000003078CC6B
:10038000CCCCFCCCCCCC000000FC6666667C6666FF
:1003900066FC0000003C66C6C0C0C0C6663C0000EB
:1003A00000F86C66666666666CF8000000FE6260C7
:1003B000647C646062FE000000FE6662647C6460CF
:1003C00060F00000003C66C6C0C0CEC6663E0000BD
:1003D00000CCCCCCCCFCCCCCCCCC000000783030E9
:1003E0003030303030780000001E0C0C0C0CCCCCBF
:1003F000CC78000000E6666C6C786C6C66E60000F9
:1004000000F060606060626666FE000000C6EEFE9E
:10041000FED6C6C6C6C6000000C6C6E6F6FEDECEDE
:10042000C6C6000000386CC6C6C6C6C66C3800001A
:1004300000FC6666667C606060F0000000386CC698
:10044000C6C6CEDE7C0C1E0000FC6666667C6C6652
:1004500066E600000078CCCCC07018CCCC780000E8
:1004600000FCB430303030303078000000CCCCCCE0
:10047000CCCCCCCCCC78000000CCCCCCCCCCCCCC74
:100480007830000000C6C6C6C6D6D66C6C6C0000BC
:1004900000CCCCCC783078CCCCCC000000CCCCCC10
:1004A000CC7830303078000000FECE981830606292
:1004B000C6FE0000003C303030303030303C0000B0
:1004C000000080C06030180C06020000003C0C0CDC
:1004D0000C0C0C0C0C3C000010386CC6000000002A
:1004E0000000000000000000000000000000FF000D
:1004F0003030180000000000000000000000000084
:10050000780C7CCCCC76000000E060607C6666668F
:1005100066DC00000000000078CCC0C0CC78000091
:10052000001C0C0C7CCCCCCCCC7600000000000075
:1005300078CCFCC0CC78000000386C6060F860605B
:1005400060F000000000000076CCCCCC7C0CCC78B5
:1005500000E060606C76666666E6000000181800D1
:1005600078181818187E0000000C0C003C0C0C0CBD
:100570000CCCCC7800E06060666C786C66E60000BD
:100580000078181818181818187E000000000000CD
:10059000FCD6D6D6D6C6000000000000F8CCCCCCE5
:1005A000CCCC00000000000078CCCCCCCC78000093
:1005B00000000000DC666666667C60F000000000FB
:1005C00076CCCCCCCC7C0C1E00000000EC6E7660AF
:1005D00060F000000000000078CC6018CC780000CB
:1005E00000002060FC6060606C38000000000000CB
:1005F000CCCCCCCCCC76000000000000CCCCCCCC59
:100600007830000000000000C6C6D6D66C6C000032
:1006100000000000C66C38386CC600000000000006
:10062000666666663C0C18F000000000FC8C1860E2
:10063000C4FC0000001C303060C06030301C000082
:1006400000181818180018181818000000E03030AA
:10065000180C183030E000000073DACE0000000003
:100660000000000000000010386CC6C6FE0000004C
:100670000078CCCCC0C0C0CCCC78306000CCCC00F2
:10068000CCCCCCCCCC7600000C18300078CCFCC0A4
:10069000CC7800003078CC00780C7CCCCC76000094
:1006A00000CCCC00780C7CCCCC760000C060300054
:1006B000780C7CCCCC760000386C6C38F80C7CCC98
:1006C000CC7600000000000078CCC0C0CC78306050
:1006D0003078CC0078CCFCC0C07C000000CCCC00D2
:1006E00078CCFCC0C07C0000C060300078CCFCC07E
:1006F000C07C0000006C6C0078181818187E000090
:1007000010386C0078181818187E00006030180037
:1007100078181818187E000000CC003078CCCCFC7B
:10072000CCCC000078CCCC7878CCCCFCCCCC000005
:100730000C1800FCC4C0F8C0C4FC0000000000009D
:10074000FE1B7FD8D8EF0000003E78D8D8FED8D85E
:10075000D8DE00003078CC0078CCCCCCCC7800004F
:1007600000CCCC0078CCCCCCCC780000C060300081
:1007700078CCCCCCCC7800003078CC00CCCCCCCCB5
:10078000CC760000C0603000CCCCCCCCCC76000065
:1007900000666600666666663C0C18F000CC007861
:1007A000CCCCCCCCCC780000CC00CCCCCCCCCCCC41
:1007B000CC7800000000000078CCDCECCC780000A5
:1007C0003C66606060FC6060C0FE0000003A6CCE79
:1007D000D6D6D6E66CB800000000000000C66C3823
:1007E0006CC600000E1B18187E181818D870000070
:1007F0000C183000780C7CCCCC7600000C18300043
:1008000078181818187E00000C18300078CCCCCC62
:10081000CC7800000C183000CCCCCCCCCC760000CE
:100820000076DC00F8CCCCCCCCCC000076DC00C66A
:10083000E6F6DECEC6C600000078CCCC7E00FE0018
:10084000000000000078CCCC7800FE000000000022
:10085000003030003060C0C0CC780000003844BAAE
:10086000AABAB2AA443800000000000000FC0C0C38
:100870000C0000000062E66C78306EC3860C1F002E
:100880000063E66C78376FDBB33F03000030300065
:100890003030787878300000000000003366CCCC2F
:1008A0006633000000000000CC66333366CC0000E5
:1008B00024924924924924924924924955AA55AA3E
:1008C00055AA55AA55AA55AA6DDBB66DDBB66DDBE8
:1008D000B66DDBB618181818181818181818181844
:1008E0001818181818F81818181818180C180030B4
:1008F00078CCCCFCCCCC000078CC003078CCCCFCD4
:10090000CCCC00006030003078CCCCFCCCCC0000EB
:10091000003844BAA2A2A2BA4438000066666666ED
:10092000E60606E666666666666666666666666627
:100930006666666600000000FE0606E66666666697
:1009400066666666E60606FE000000000030307847
:10095000CCC0C0CC78303000CCCCCCCC78FC30FCD7
:10096000303000000000000000F81818181818189F
:1009700018181818181F0000000000001818181880
:1009800018FF0000000000000000000000FF181821
:100990001818181818181818181F181818181818D0
:1009A0000000000000FF00000000000018181818E8
:1009B00018FF1818181818180076DC00780C7CCC72
:1009C000CC76000076DC003078CCCCFCCCCC0000BF
:1009D000666666666760607F0000000000000000D9
:1009E0007F6060676666666666666666E70000FF4B
:1009F0000000000000000000FF0000E76666666679
:100A00006666666667606067666666660000000028
:100A1000FF0000FF0000000066666666E70000E772
:100A2000666666660000000000C67C6C7CC600003E
:100A3000CC30D80C067EC6C6C67C000000F86C66BA
:100A400066F666666CF8000078CC00FCC4C0F8C09E
:100A5000C4FC000000CC00FCC4C0F8C0C4FC000012
:100A6000603000FCC4C0F8C0C4FC000000F03030AE
:100A700030FC0000000000001830007830303030CA
:100A80003078000078CC007830303030307800009A
:100A900000CC00783030303030780000181818184A
:100AA00018F800000000000000000000001F1818E7
:100AB00018181818FFFFFFFFFFFFFFFFFFFFFFFFE2
:100AC000000000000000FFFFFFFFFFFF00181818E4
:100AD00018001818181800006030007830303030D6
:100AE00030780000FFFFFFFFFFFF00000000000064
:100AF00018300078CCCCCCCCCC7800000078CCCCB2
:100B0000D8CCCCCCF8C0600078CC0078CCCCCCCCA5
:100B1000CC78000060300078CCCCCCCCCC78000015
:100B20000076DC0078CCCCCCCC78000076DC007889
:100B3000CCCCCCCCCC7800000000000066666666A9
:100B4000667B60C00000E0607C66667C60F0000050
:100B500000F0607C6666667C60F00000183000CCB7
:100B6000CCCCCCCCCC78000078CC00CCCCCCCCCCD1
:100B7000CC780000603000CCCCCCCCCCCC78000061
:100B8000060C1800666666663C0C18F0183000CC3F
:100B9000CCCC78303078000000FC00000000000071
:100BA000000000000C1830000000000000000000F1
:100BB0000000000000FC00000000000000003030D9
:100BC000FC303000FC0000000000000000F80000D5
:100BD000F8000000E033663CF8376FDBB33F0300FA
:100BE000007FDBDBDB7B1B1B1B1B0000007E6330FD
:100BF0003C66663C0CC67E000000303000FC0030D5
:100C00003000000000000000000000000000307014
:100C1000003C6666663C00000000000000CC00005E
:100C200000000000000000000000000000180000AC
:100C3000000000000030703030780000000000003C
:100C400000780C380C7800000000000000780C18C8
:100C5000307C000000000000000000FCFCFCFCFCFC
:100C6000FC00000000000000000000000000000088
:100C70003820636F6C6F7572206D6F6465206279C8
:100C80002053656261737469616E00B820627920D7
:100C900042656E6564696B7400333230783234308B
:100CA000204C434420436F6E74726F6C6C6572000D
:100CB00011241FBECFEFD4E0DEBFCDBF11E0A0E016
:100CC000B1E0EEE6F0E202C005900D92A230B1076D
:100CD000D9F712E0A2E0B1E001C01D92A13DB10739
:100CE000E1F70E9477060C9435100C9400008FEF0A
:100CF0008BBB85BB97E092BB87BB9EEF91BB86B950
:100D00000E94DD0B82E290E061E00E948B0D10E01A
:100D1000C0E0D0E088248A9499240CE0302EB4E618
:100D20002B2E0E949D0D482F803208F067C0813025
:100D300009F479C0823009F47AC0833009F479C0AB
:100D4000883009F478C0893009F48CC08A3009F4FD
:100D500083C08B3009F472C08C3009F49EC08D3092
:100D600009F444C08E3009F4A2C08F3009F4A2C047
:100D7000803109F4B3C0813109F4F1C0823109F442
:100D800008C1833109F425C1853109F43DC186319B
:100D900009F441C1893109F445C18B3109F487C097
:100DA0008C3109F484C08D3109F457C18E3109F0BA
:100DB000B8CF0E949D0D882309F072C10E949D0D3D
:100DC000482FCE0196958795969587959695879508
:100DD000612F282D092D0E9482082896F1E0C03449
:100DE000DF0708F49ECF145F103FE8F4C0E0D0E0C6
:100DF0000E949D0D482F803208F499CFCE01969520
:100E000087959695879596958795612F282D092D1D
:100E10000E94E50F289681E0C034D80708F481CFFE
:100E2000145F103F18F310E0C0E0D0E07ACF38989C
:100E300078CF389A76CF2897D7FD27C0CE019695E0
:100E400087959695879596958795612F40E2282DF1
:100E5000092D0E94E50F65CF145F103F08F461CFA4
:100E600010E05FCF0E949D0DF82E0E949D0D082F6F
:100E70000E949D0DE82E0E949D0D482F8F2D902FD2
:100E80006E2D70E00E94F60E4CCF1C50103F58F0B3
:100E900014EEC8E3D1E087E2D8CF0E94730810E0D7
:100EA000C0E0D0E03ECFC8E3D1E087E2CECF0E94E1
:100EB0009D0D37CF0E949D0D90E0A0E0B0E0BC01F9
:100EC000CD012AE932E040E050E00E941610672F81
:100ED000782F892F992779BD68BD23CF0E949D0D5A
:100EE0008A3A09F01ECF0E949D0D482E0E949D0D4A
:100EF000D82E0E949D0D582E0E949D0D682E0E9496
:100F00009D0D782E662009F40CCFAA24552011F1EE
:100F1000E42CCC2420924F0205C080914F028823FC
:100F200009F4FFCE0E94BA0D892BB9F30E949D0DE2
:100F3000F82E91E0791609F4D0C0E2E07E1609F4AB
:100F4000BFC08E2D6D2D4F2D0E94380FC394E3949A
:100F5000C51400F3A394D394A614C0F2E2CE0E9469
:100F60009D0DC82FD0E0CC0FDD1FCC0FDD1FCC0FA7
:100F7000DD1F0E949D0D839D102D1124F1E0C034D2
:100F8000DF0710F0C0E0D0E0103F08F4CACE10E058
:100F9000C8CE0E949D0DE82E0E949D0DD82E0E9465
:100FA0009D0DC82E0E949D0DB82E0E949D0DA82E4D
:100FB0000E949D0DF82E0E949D0D082F8E2D9D2DB7
:100FC0006C2D70E04B2D5A2D2F2D30E00E94D4094E
:100FD000A8CE0E949D0DC82E0E949D0DB82E0E9485
:100FE0009D0DF82E0E949D0DE82E0E949D0DD82E7D
:100FF0000E949D0D082F8C2D9B2D6F2D70E04E2D86
:101000002D2D0E94760A8DCE0E949D0D882E0E9465
:101010009D0D982E86CE0E949D0D0E949D0D0E94D2
:101020009D0D7FCE0E949D0DE82EFF2487E0E822D3
:10103000FF24EE0CFF1CEE0CFF1CEE0CFF1CE1E588
:10104000F2E0EE0EFF1E00E00E949D0DF70181937D
:101050007F010F5F0830C1F764CE0E949D0D782E8E
:101060000E949D0DF82E0E949D0DD82E0E949D0D70
:10107000C82E0E949D0DB82E0E949D0DA82E0E9484
:101080009D0D082F0E949D0DE82E872D9F2D6D2D03
:1010900070E04C2D5B2D2A2D30E00E94190A41CEC4
:1010A0000E949D0D482FCE01969587959695879520
:1010B00096958795612F282D092D0E94E50F8DCEDD
:1010C0000E949D0DB82E0E949D0D082F8E2D6D2D16
:1010D0004F2D2B2D0E94810F39CF8E2D6D2D4F2D31
:1010E0000E94460F33CFE0E0F5E011923097E9F728
:1010F0000895893108F088E190E0880F991F809366
:10110000500208955F926F927F928F929F92AF925A
:10111000BF92CF92DF92EF92FF920F931F93782EA0
:10112000162FE42E622E8FE0E822FF2461E5862E42
:1011300062E0962EEE0CFF1CEE0CFF1CEE0CFF1C6A
:101140006401CE0CDF1C872D612FF60140810E94C7
:10115000C00F1F5F872D612FF6014081262D0E9451
:10116000C00F1F5F872D612FF6014181262D0E9440
:10117000C00F1F5F82E090E0E80EF91E5401AE0C34
:10118000BF1CEEEFFFEFEE0EFF1E872D612FF50166
:101190004081262D0E94C00F1F5F872D612FF50112
:1011A0004081262D0E94C00F1F5F872D612FF60101
:1011B0004381262D0E94C00F1F5F8E0C9F1C872D20
:1011C000612FF4014481262D0E94C00F1F5F872DDF
:1011D000612FF6014581262D0E94C00F1F5F872DCC
:1011E000612FF6014581262D0E94C00F1F5F872DBC
:1011F000612FF6014681262D0E94C00F1F5F872DAB
:10120000612FF6014781262D0E94C00F1F5F872D99
:10121000612FF6014781262D0E94C00F1F910F916B
:10122000FF90EF90DF90CF90BF90AF909F908F9006
:101230007F906F905F9008952F923F924F925F92B0
:101240006F927F928F929F92AF92BF92CF92DF92D6
:10125000EF92FF920F931F93DF93CF9300D00F92E3
:10126000CDB7DEB77C012B014A015901302E881A17
:10127000990AA61AB70A181419040CF08EC081E056
:1012800089831A141B040CF081C022242394C70103
:10129000B201432D0E94F60E8A149B040CF046C046
:1012A000A114B10469F1F401EE0FFF1FFB83EA837F
:1012B000622C772467FC70946701720100E010E0F3
:1012C000F9814F2E552447FC50948A819B81880DCB
:1012D000991D9B838A838A159B0534F08A199B0983
:1012E0009B838A83C40CD51CE60CF71CC601B7018E
:1012F000432D0E94F60E0F5F1F4F0A151B0528F3A2
:101300000F900F900F90CF91DF911F910F91FF9051
:10131000EF90DF90CF90BF90AF909F908F907F9095
:101320006F905F904F903F902F900895811491049B
:1013300039F3F501EE0FFF1FFB83EA83F9816F2E6E
:10134000772467FC7094620100E010E0422C552481
:1013500047FC50948A819B818A0D9B1D9B838A83C5
:101360008815990534F0881999099B838A83C40CE0
:10137000D51CE60CF71CC701B601432D0E94F60EE2
:101380000F5F1F4F0815190528F3BACFB094A19429
:10139000B108B39422242A947ACF9094819491082E
:1013A00093949FEF99836DCF8F929F92AF92BF924C
:1013B000CF92DF92EF92FF920F93CF93DF934C0186
:1013C0006B015A01790162177307F9F084179507C9
:1013D00071F00E941C09DF91CF910F91FF90EF9067
:1013E000DF90CF90BF90AF909F908F900895261779
:1013F0003707C8F0E601C401BE01402F0E94F60E77
:101400002196EC16FD06B8F7E6CF4817590770F09D
:10141000E401CE01B601402F0E94F60E2196AC16D3
:10142000BD06B8F7D8CF7B016901E4CF4A015C0162
:10143000EFCF3F924F925F926F927F928F929F92E7
:10144000AF92BF92CF92DF92EF92FF920F931F93D2
:10145000CF93DF933C012B014A016901102F3E2CF1
:101460005C010894A11CB11CA416B506A0F4EB0104
:101470002196C217D30778F47A010894E108F1089D
:10148000C501BE01A7019E01012F0E94D40921962A
:10149000CC15DD05A8F3C301B201A4019201032D0F
:1014A0000E94D409C401B201A40196010E94D4098A
:1014B000C401B601A30196010E94D409C301B6017B
:1014C000A30192010E94D409DF91CF911F910F9146
:1014D000FF90EF90DF90CF90BF90AF909F908F9054
:1014E0007F906F905F904F903F9008952F923F9222
:1014F0004F925F926F927F928F929F92AF92BF9224
:10150000CF92DF92EF92FF920F931F93DF93CF93CF
:10151000CDB7DEB72C970FB6F894DEBF0FBECDBFA8
:101520002C011B014987122F0A87642E7724861508
:10153000970508F483C06615770508F47FC0442337
:1015400009F47CC0842F90E0880F991F222733274D
:10155000281B390B2D5F3F4F3A83298348878980A9
:101560009A807C866B86AA24BB241D821C8224C0A0
:10157000288521502887822F90E09C878B87EAE07E
:10158000F0E08E0E9F1EC5012B853C85821B930BC0
:10159000880F991F880F991F880E991E0894A11C07
:1015A000B11C8C819D8104969D838C83EB85FC8589
:1015B000EA15FB0508F45BC07201EA18FB08650137
:1015C000C40CD51C2B853C85220D331DC701B901E8
:1015D000A601012F0E94D40991018B859C85281BAF
:1015E000390BC701B901A6010E94D4097201EB852C
:1015F000FC85EE1AFF0A6F01C40CD51C9501220D63
:10160000331DC701B901A6010E94D40991012A190D
:101610003B09C701B901A6010E94D40997FEA8CFD2
:101620002C813D81820E931E86E090E0880E991EEB
:10163000F885EF2FF0E0FC87EB87B0CF2C960FB644
:10164000F894DEBF0FBECDBFCF91DF911F910F91F8
:10165000FF90EF90DF90CF90BF90AF909F908F90D2
:101660007F906F905F904F903F902F900895F985F5
:10167000FB831C861B861F821E8223C08B818150A8
:101680008B83682E7724E981FA813A968B859C8535
:1016900086199709880F991F880F991FE80FF91F5E
:1016A000FA83E9832B853C852F5F3F4F3C872B874F
:1016B0008E819F8104969F838E836216730608F441
:1016C000BDCFEB84FC84E40CF51C4301820C931C1D
:1016D000C701B4014A850E94F60E8301040D151D51
:1016E000AB84BC84A20CB31CC801B5014A850E941E
:1016F000F60E61012B853C85C21AD30AC801B601DA
:101700004A850E94F60E810106191709C701B80122
:101710004A850E94F60E72018B859C85E81AF90AAB
:10172000C701B8014A850E94F60E82010619170901
:10173000C801B6014A850E94F60EC801B5014A8566
:101740000E94F60EC701B4014A850E94F60EE98197
:10175000FA81F7FF93CF2E813F812E0F3F1F2A5F23
:101760003F4F3A8329833B81632E77249BCFDF92BF
:10177000EF92FF920F931F93CF93DF93D62EFA0130
:10178000E22EF02E4491442381F0EF01219601C016
:10179000812F182F1F5F6D2D2E2D0F2D0E94E50F0D
:1017A000FE0121964491442399F7DF91CF911F9137
:1017B0000F91FF90EF90DF900895EF920F93CF93EA
:1017C000DF93F89488E10FB6F89481BD11BC0FBE89
:1017D00080E885BF8AE090E09BBD8ABD8DE491E002
:1017E00099BD88BD89E992E095BD84BD82EB8FBD2E
:1017F00089E18EBD89B7806889BF7894E0E0F5E023
:1018000011923097E9F782E390E06AE070E04DE0F2
:1018100051E02FE430E000E0EE24EA940E94190A3F
:101820008CE390E064E170E04DE650E025E430E0C8
:1018300000E40E94190A86E990E06FE070E04DEB49
:1018400050E02DE230E0F0E4EF2E0E94190A84EB24
:1018500090E068E270E04BED50E02BE430E000E80F
:10186000E0E8EE2E0E94190A88EC90E064E170E056
:101870004FEE50E022E330E00FEFEE24EA940E94B6
:10188000190AE9E9FCE04491442389F0EF0121962B
:101890008AE001C08E2DE82EE39468E72FEF00E088
:1018A0000E94E50FFE0121964491442399F7EBE84D
:1018B000FCE04491442389F0EF0121968FE001C0C0
:1018C0008E2DE82EE3946CE82FEF00E00E94E50FE8
:1018D000FE0121964491442399F7E0E7FCE044910E
:1018E000442389F0EF01219687E001C08E2DE82E78
:1018F000E39468EC2FEF00E00E94E50FFE012196D3
:101900004491442399F780E090E067ED70E043E173
:1019100050E02CED30E00FEFEE24EA940E94190A1B
:1019200084E190E067ED70E047E250E02CED30E0BC
:1019300000ECB0ECEB2E0E94190A88E290E067ED13
:1019400070E04BE350E02CED30E000EAA0EAEA2E34
:101950000E94190A8CE390E067ED70E04FE450E0DC
:101960002CED30E000E8F0E8EF2E0E94190A80E547
:1019700090E067ED70E043E650E02CED30E000E6EB
:10198000E0E6EE2E0E94190A84E690E067ED70E032
:1019900047E750E02CED30E000E4B0E4EB2E0E948D
:1019A000190A88E790E067ED70E04BE850E02CED15
:1019B00030E000E2A0E2EA2E0E94190A8CE890E0F2
:1019C00067ED70E04FE950E02CED30E000E0EE24F0
:1019D0000E94190A80EA90E067ED70E043EB50E066
:1019E0002CED30E00E94190A84EB90E067ED70E086
:1019F00047EC50E02CED30E000E2F0E2EF2E0E94E8
:101A0000190A88EC90E067ED70E04BED50E02CEDAA
:101A100030E000E4E0E4EE2E0E94190A8CED90E044
:101A200067ED70E04FEE50E02CED30E000E6B0E600
:101A3000EB2E0E94190A80EF90E067ED70E043E022
:101A400051E02CED30E000E8A0E8EA2E0E94190AEF
:101A500084E091E067ED70E047E151E02CED30E08B
:101A600000EAF0EAEF2E0E94190A88E191E067EDA2
:101A700070E04BE251E02CED30E000ECE0ECEE2EBB
:101A80000E94190A8CE291E067ED70E04FE351E0AB
:101A90002CED30E00FEFEE24EA940E94190A2CE0BE
:101AA00088E190E00FB6F894A89581BD0FBE21BDE6
:101AB000389ADF91CF910F91EF9008951F920F9276
:101AC0000FB60F9211248F939F93EF93FF939CB1C6
:101AD000E0910202EF5F80910302E81799F0E09332
:101AE0000202F0E0EE5FFE4F90838091040290913D
:101AF000050201969093050280930402813C9105B2
:101B000008F0929AFF91EF919F918F910F900FBEE5
:101B10000F901F9018951092020210920302929853
:101B2000109205021092040290BD89B96111599A70
:101B300080E98AB986E880BD0895E091030280912A
:101B400002028E17E1F3EF5FE0930302F8948091B5
:101B5000040290910502019790930502809304027C
:101B6000803C910508F492987894F0E0EE5FFE4F87
:101B7000808108952091040230910502C9010895E1
:101B80001F920F920FB60F9211242F938F939F9352
:101B9000EF93FF9392B123B1E0914802EF5FEF71B1
:101BA00080914902E817A1F0892F8871E0934802DB
:101BB000F0E0EA5DFD4F208380934A02FF91EF91B0
:101BC0009F918F912F910F900FBE0F901F9018959E
:101BD00082E0F2CF1F920F920FB60F9211248F93D3
:101BE0009F93EF93FF93909146028091470298173D
:101BF000A1F0E0914702EF5FEF71E0934702F0E060
:101C0000EA5FFD4F808183B9FF91EF919F918F91A2
:101C10000F900FBE0F901F9018950D98F5CF109252
:101C200046021092470210924802109249029CBF4D
:101C300080B988E981B986E88CBF089590914802FF
:101C4000809149029817A1F0E0914902EF5FEF718E
:101C5000E0934902F0E0EA5DFD4F308120914A02B5
:101C6000922F80E0AC01430F511D9A01C9010895E4
:101C700020E031E0C9010895282F909146029F5F2E
:101C80009F71809147029817E1F3E92FF0E0EA5F36
:101C9000FD4F2083909346020D9A0895CF93DF93D2
:101CA000EC018881882331F021960E943C0E8881C6
:101CB0008823D1F7DF91CF910895CF93DF93FC0173
:101CC0008491882349F0EF0121960E943C0EFE0189
:101CD000219684918823C9F7DF91CF9108950F93BE
:101CE0000FB70F93AF93BF932F9320914E02AA2764
:101CF00021FF03C0A05B20FDA05B2D5F273008F013
:101D0000275020934E02B0914C02B39594980D91B8
:101D10000D910D910D910D910D910D910D910D91D3
:101D20000D910D910D910D910D910D910D910D91C3
:101D30000D910D910D910D910D910D910D910D91B3
:101D40000D910D910D910D910D910D910D910D91A3
:101D50000D910D910D910D910D910D910D910D9193
:101D60000D910D910D910D910D910D910D910D9183
:101D70000D910D910D910D910D910D910D910D9173
:101D80000D910D910D910D910D910D910D910D9163
:101D90000D910D910D910D910D910D910D910D9153
:101DA0000D910D910D910D910D910D910C91B530FD
:101DB00089F4949AA89520914F022A9520934F0276
:101DC00020914D022395273008F0222720934D02C1
:101DD00020934E02B53F08F0B4E0B0934C022F912F
:101DE000BF91AF910F910FBF0F91189521E08A3AE3
:101DF0009207E8F5603FD8F5582F577030E850301B
:101E000019F036955A95E9F79695879596958795A1
:101E1000A82FB62FBB5FF894939A5C91939878940F
:101E200047FF03C0532B5C9304C0309553235C934E
:101E30003095A05BF894939A5C919398789446FFC0
:101E400003C0532B5C9304C0309553235C933095AF
:101E5000A05BF894939A5C919398789445FF03C0A3
:101E6000532B5C9304C0309553235C9330950895B5
:101E7000853358F4603F48F4A82FAA0FB62FBB5FF4
:101E80004C93A05B4C93A05B4C9308958A36C0F5AD
:101E9000603FB0F5A82FB62FBB5F55276627441FBC
:101EA000551F441F661F441F551F441F661F441FB4
:101EB000551F441F661F441F551F441F661F70EFA8
:101EC000A0FF7295A0FF5295F894939A4C91939825
:101ED00078944723542B5C93A0FF6295A05BF89401
:101EE000939A4C91939878944723642B6C93A05BBE
:101EF000F894939A4C91939878944723642B6C931D
:101F000008958533E0F5603FD0F5A82FAA0FB62FCE
:101F1000BB5F441F331F441F551F441F771F441FBF
:101F2000331F441F551F441F771F441F331F441F77
:101F3000551F221F771F221F331F221F551F221FCD
:101F4000771F221F331F221F551F221F771F221F9B
:101F5000331F402F441F551F441F771F441F331F3B
:101F6000441F551F441F771F441F331F441F551F15
:101F7000441F771F3C93A05B5C93A05B7C93089508
:101F8000853310F5603F00F5880FB62FBB5F902FAB
:101F90009223202B642FA82F07FD409527FF44276D
:101FA00097FD4FEF4C93462FA05B06FD609526FFF3
:101FB000662796FD6FEF6C93A05B05FD409525FFAE
:101FC000442795FD4FEF4C930895853370F5603F9E
:101FD00060F5E42FFCE0EF9FF001E059FF4F5CE07B
:101FE000880FB62FBB5F902F9223202B4591642F33
:101FF000A82F07FD409527FF442797FD4FEF4C93EF
:10200000462FA05B06FD609526FF662796FD6FEFC5
:102010006C93A05B05FD409525FF442795FD4FEF90
:102020004C93B3955A9511F711240895629FD001EE
:10203000739FF001829FE00DF11D649FE00DF11D83
:10204000929FF00D839FF00D749FF00D659FF00D32
:102050009927729FB00DE11DF91F639FB00DE11D1F
:0E206000F91FBD01CF0111240895F894FFCFA0
:02206E0000056B
:00000001FF
